:100000002820002001010000FD000000FD0000008C
:1000100000000000000000000000000000000000E0
:10002000000000000000000000000000FD000000D3
:100030000000000000000000FD000000FD000000C6
:10004000FD000000FD000000FD000000FD000000BC
:10005000FD000000FD000000FD000000FD000000AC
:10006000FD000000FD000000FD000000FD0000009C
:10007000FD000000FD000000FD000000FD0000008C
:10008000FD000000FD000000FD000000FD0000007C
:10009000FD000000FD000000FD000000FD0000006C
:1000A000FD000000FD000000FD000000FD0000005C
:1000B0000000000010B5064C2378002B07D1054B3B
:1000C000002B02D0044800E000BF0123237010BDC4
:1000D000000000200000000034060000044B10B5B2
:1000E000002B03D00349044800E000BF10BDC04608
:1000F000000000000400002034060000FEE70000BD
:100100002549264870B581420AD0254BC41E0022DD
:10011000A34203D303331A1A92089200214B984743
:100120002148224BC11E0022994203D803331A1AD8
:100130009208920000211E4B9847FF221D4B03217D
:1001400093431D4A0C2593600222082430261B4B42
:100150001B485A62C3788B431343C370C378AB43C5
:100160002343C370174B987BB043060020203043D5
:100170009873987BA84304439C73987B88430243FD
:100180009A738023104A51680B4353600F4B984772
:100190000F4B9847FEE7C0463406000000000020E1
:1001A00000000020B9050000000000202800002009
:1001B000CB0500000000000000ED00E0FC700041F5
:1001C000005000410048004100400041710500001E
:1001D000B5030000064B1A7AD2B21A725A7AD2B21A
:1001E0005A729A7AD2B29A72DA7AD2B2DA727047C4
:1001F00000040040064B10B55A685A60054B9847FA
:10020000054B9847054B9847FF20054B984710BD75
:1002100000400041D50100002D02000075020000E1
:1002200095030000002800D100BE70470E4B186AED
:10023000196A890F8A070D4901400A430C490A438C
:100240001A62022299690A431F219A611A7F0A40A1
:100250001A771E39DA68D2080A42FBD08022196A5E
:100260000A431A627047C046000800400000FF0FB2
:10027000020300000221024A93698B439361704795
:1002800000080040F8B506000D001400002804D056
:10029000081E02D01000431E9841F1221049114B54
:1002A00098473700083738000F4B98470028F8D098
:1002B00000263800A95D0D4B984738000A4B984737
:1002C0000028FAD00136B442F3D80125002C00D022
:1002D00025003800064B98470028FAD02800F8BDC2
:1002E000DA0500002502000047050000390500007E
:1002F00051050000F7B5050014000191002804D055
:10030000081E02D01000431E984186220C490D4B56
:100310005200984700262F00083738000A4B9847AC
:100320000028F8D0094B38009847019B98550136B2
:10033000B442F0D80120002C00D02000FEBDC04601
:10034000DA050000250200005B0500003F05000003
:1003500070B504000D00002802D00800431E98412B
:100360000749084B3422984720002900064B0830E3
:100370009847002803D1054B6360054B236070BD8F
:10038000DA050000250200000D050000F50200005E
:1003900085020000C30709D58023054A5B009360EE
:1003A00083235B0253605378DB09FCD17047C0465E
:1003B000000C004010B5014B9847FEE765050000B2
:1003C0000D4B0122180030B5443001780F249143C1
:1003D000114301701900032032310D784533A543D4
:1003E000284308701878904302431A700B781C4019
:1003F000302323430B7030BD004400410423044AE2
:10040000116A0B431362034B034A5A807047C0467C
:1004100000040040000C00401440000010B5054BE3
:10042000984700220449054B05489847054B9847D3
:1004300010BDC046FD03000000080042510300004B
:100440001C000020C103000010B5024B9847024B6E
:10045000984710BDF50100001D040000C369194252
:10046000FCD17047022210B5036803219343036057
:10047000014B984710BDC0465D0400001B4B70B592
:10048000C3189B0ADBB20400002B04D00020184ADA
:100490001849194B9847E369184DDB0711D4022618
:1004A00003212000A8472368334205D02000144BC5
:1004B000984731002000A84705230321200023602E
:1004C000A84720000121A8470E4B200023600321EC
:1004D000A847C0239B02200063600721A847002093
:1004E000094BA381A0733034207070BD00F8FFBDAC
:1004F0003A020000F6050000250200005D0400003D
:100500006504000004001040ADD8FFFF70B5050081
:10051000431E98410C00B4220449054BC0B29847D1
:100520002C602000034B984770BDC046F6050000C4
:10053000250200007D0400000368198570470368E8
:10054000188DC0B270470368187E012318407047A9
:100550000368187E8007C00F70470368187E400745
:10056000C00F704710B5014B984710BD49040000FB
:1005700070B500260C4D0D4C641BA410A64209D189
:10058000002600F047F80A4D0A4C641BA410A6424E
:1005900005D170BDB300EB5898470136EEE7B300C4
:1005A000EB5898470136F2E72006000020060000CD
:1005B0002006000024060000002310B59A4200D156
:1005C00010BDCC5CC4540133F8E703008218934299
:1005D00000D1704719700133F9E72E2E2F68616C36
:1005E0002F7372632F68616C5F75736172745F73D0
:1005F000796E632E63002E2E2F68706C2F736572D8
:10060000636F6D2F68706C5F736572636F6D2E63BF
:1006100000000000F8B5C046F8BC08BC9E46704714
:10062000DD000000F8B5C046F8BC08BC9E46704727
:04063000B500000011
:00000001FF
